ARM GAS  C:\Cache\ccCtM5Kc.s 			page 1


   1              		.syntax unified
   2              		.cpu cortex-m3
   3              		.fpu softvfp
   4              		.eabi_attribute 20, 1
   5              		.eabi_attribute 21, 1
   6              		.eabi_attribute 23, 3
   7              		.eabi_attribute 24, 1
   8              		.eabi_attribute 25, 1
   9              		.eabi_attribute 26, 1
  10              		.eabi_attribute 30, 1
  11              		.eabi_attribute 34, 1
  12              		.eabi_attribute 18, 4
  13              		.thumb
  14              		.syntax unified
  15              		.file	"main.c"
  16              		.text
  17              	.Ltext0:
  18              		.cfi_sections	.debug_frame
  19              		.section	.text.main,"ax",%progbits
  20              		.align	2
  21              		.global	main
  22              		.thumb
  23              		.thumb_func
  24              		.type	main, %function
  25              	main:
  26              	.LFB64:
  27              		.file 1 "main.c"
   1:main.c        **** /* Emilio MARITON BTS 951 17/11/2021 */
   2:main.c        **** 
   3:main.c        **** //(00 58 13 AD E6) ID à obtenir
   4:main.c        **** 
   5:main.c        **** #include "project.h"
   6:main.c        **** #include "stdio.h"
   7:main.c        **** 
   8:main.c        **** 
   9:main.c        **** 
  10:main.c        **** int main(void)
  11:main.c        **** {
  28              		.loc 1 11 0
  29              		.cfi_startproc
  30              		@ Volatile: function does not return.
  31              		@ args = 0, pretend = 0, frame = 0
  32              		@ frame_needed = 0, uses_anonymous_args = 0
  33 0000 08B5     		push	{r3, lr}
  34              		.cfi_def_cfa_offset 8
  35              		.cfi_offset 3, -8
  36              		.cfi_offset 14, -4
  12:main.c        ****     CyGlobalIntEnable; //Active toutes les interuptions
  37              		.loc 1 12 0
  38              		.syntax unified
  39              	@ 12 "main.c" 1
  40 0002 62B6     		CPSIE   i
  41              	@ 0 "" 2
  13:main.c        ****     UART_Start();//Initialise le bloc UART
  42              		.loc 1 13 0
  43              		.thumb
  44              		.syntax unified
ARM GAS  C:\Cache\ccCtM5Kc.s 			page 2


  45 0004 FFF7FEFF 		bl	UART_Start
  46              	.LVL0:
  14:main.c        ****     rfid_Start();
  47              		.loc 1 14 0
  48 0008 FFF7FEFF 		bl	rfid_Start
  49              	.LVL1:
  15:main.c        ****     UART_PutString("Fin Init");//Informe de la fin de la phase d'initialisation
  50              		.loc 1 15 0
  51 000c 0148     		ldr	r0, .L4
  52 000e FFF7FEFF 		bl	UART_PutString
  53              	.LVL2:
  54              	.L2:
  55 0012 FEE7     		b	.L2
  56              	.L5:
  57              		.align	2
  58              	.L4:
  59 0014 00000000 		.word	.LC0
  60              		.cfi_endproc
  61              	.LFE64:
  62              		.size	main, .-main
  63              		.section	.rodata.str1.4,"aMS",%progbits,1
  64              		.align	2
  65              	.LC0:
  66 0000 46696E20 		.ascii	"Fin Init\000"
  66      496E6974 
  66      00
  67              		.text
  68              	.Letext0:
  69              		.file 2 "c:\\program files (x86)\\cypress\\psoc creator\\4.2\\psoc creator\\import\\gnu\\arm\\5.4.
  70              		.file 3 "c:\\program files (x86)\\cypress\\psoc creator\\4.2\\psoc creator\\import\\gnu\\arm\\5.4.
  71              		.file 4 "Generated_Source\\PSoC5/UART.h"
  72              		.file 5 "Generated_Source\\PSoC5/rfid.h"
  73              		.file 6 "Generated_Source\\PSoC5/core_cm3.h"
